Archive member included       because of file (symbol)

C:\PROGRA~1\CYGNUS\THUMBELF-000512\H-I686-CYGWIN32\BIN/../lib/gcc-lib/thumb-elf/2.9-arm-000512/libgcc.a(_call_via_rX.o)
                              main.o (_call_via_r0)
C:\PROGRA~1\CYGNUS\THUMBELF-000512\H-I686-CYGWIN32\BIN/../lib/gcc-lib/thumb-elf/2.9-arm-000512/libgcc.a(_divsi3.o)
                              main.o (__divsi3)
C:\PROGRA~1\CYGNUS\THUMBELF-000512\H-I686-CYGWIN32\BIN/../lib/gcc-lib/thumb-elf/2.9-arm-000512/libgcc.a(_dvmd_tls.o)
                              C:\PROGRA~1\CYGNUS\THUMBELF-000512\H-I686-CYGWIN32\BIN/../lib/gcc-lib/thumb-elf/2.9-arm-000512/libgcc.a(_divsi3.o) (__div0)

Allocating common symbols
Common symbol       size              file

Oam                 0x480             main.o
hz                  0x4               main.o
player              0x48              player.o
v_phase             0x4               main.o
Sky                 0x34              bg.o
Cont                0x4               main.o
state               0x4               main.o
DisplayArea         0x4               bg.o
rasttable           0x100             main.o
Light               0x34              bg.o
Trg                 0x4               main.o
player_awa          0x60              player.o
wave2nd             0xc               bg.o
OceanA              0x34              bg.o
fukiya              0x40              enemy.o
sora_xPos           0x4               bg.o
counter             0x4               main.o
IntrMainBuf         0x800             main.o
Sango_ScreenDat     0x800             bg.o
UmiA_ScreenDat      0x800             bg.o
amp_r               0x4               main.o
IntrCheck           0x4               main.o
offset              0x4               main.o
Bg2_ScreenDat       0x800             bg.o
ring                0x280             ring.o
Coral               0x34              bg.o
OceanB              0x34              bg.o
awa                 0x140             enemy.o
ocean_xPos          0x4               bg.o
Sky_ScreenDat       0x800             bg.o
dEnemy              0x2f8             enemy.o

Memory Configuration

Name             Origin             Length             Attributes
*default*        0x00000000         0xffffffff

Linker script and memory map

LOAD crt0.o
LOAD main.o
LOAD player.o
LOAD player_dat.o
LOAD enemy.o
LOAD enemy_dat.o
LOAD game_dat.o
LOAD bg.o
LOAD hitcheck.o
LOAD ring.o
LOAD obj/r_kihon0.o
LOAD obj/r_kihon1.o
LOAD obj/r_kihon2.o
LOAD obj/r_kihon3.o
LOAD obj/r_kihon4.o
LOAD obj/r_kihon5.o
LOAD obj/r_kihon6.o
LOAD obj/r_kihon7.o
LOAD obj/r_up0.o
LOAD obj/r_up1.o
LOAD obj/r_up2.o
LOAD obj/r_up3.o
LOAD obj/r_up4.o
LOAD obj/r_up5.o
LOAD obj/r_up6.o
LOAD obj/r_up7.o
LOAD obj/r_up8.o
LOAD obj/r_go_up0.o
LOAD obj/r_go_up1.o
LOAD obj/r_go_up2.o
LOAD obj/r_go_up3.o
LOAD obj/r_go_up4.o
LOAD obj/r_go_up5.o
LOAD obj/r_go_up6.o
LOAD obj/r_go_up7.o
LOAD obj/r_down0.o
LOAD obj/r_down1.o
LOAD obj/r_down2.o
LOAD obj/r_down3.o
LOAD obj/r_down4.o
LOAD obj/r_down5.o
LOAD obj/r_down6.o
LOAD obj/r_down7.o
LOAD obj/r_down8.o
LOAD obj/r_go_down0.o
LOAD obj/r_go_down1.o
LOAD obj/r_go_down2.o
LOAD obj/r_go_down3.o
LOAD obj/r_go_down4.o
LOAD obj/r_go_down5.o
LOAD obj/r_go_down6.o
LOAD obj/r_go_down7.o
LOAD obj/r_jump0.o
LOAD obj/r_jump1.o
LOAD obj/r_jump2.o
LOAD obj/r_jump3.o
LOAD obj/r_jump4.o
LOAD obj/r_jump5.o
LOAD obj/r_jump6.o
LOAD obj/r_jump7.o
LOAD obj/r_jump8.o
LOAD obj/r_jump9.o
LOAD obj/r_jump10.o
LOAD obj/r_attack1.o
LOAD obj/r_attack2.o
LOAD obj/r_attack3.o
LOAD obj/r_attack4.o
LOAD obj/r_attack5.o
LOAD obj/r_attack6.o
LOAD obj/r_attack7.o
LOAD obj/o_kihon001.o
LOAD obj/o_kihon002.o
LOAD obj/o_kihon003.o
LOAD obj/o_kihon004.o
LOAD obj/o_kihon005.o
LOAD obj/o_kihon006.o
LOAD obj/o_kihon007.o
LOAD obj/o_kihon008.o
LOAD obj/o_kihon009.o
LOAD obj/o_kihon010.o
LOAD obj/o_kougeki000.o
LOAD obj/o_kougeki001.o
LOAD obj/o_kougeki002.o
LOAD obj/o_kougeki003.o
LOAD obj/o_kougeki004.o
LOAD obj/o_kougeki005.o
LOAD obj/o_kougeki006.o
LOAD obj/o_kougeki007.o
LOAD obj/o_kougeki008.o
LOAD obj/o_kougeki009.o
LOAD obj/o_kougeki010.o
LOAD obj/o_kougeki011.o
LOAD obj/o_kougeki012.o
LOAD obj/o_kougeki013.o
LOAD obj/o_kougeki014.o
LOAD obj/o_kougeki015.o
LOAD obj/o_kougeki016.o
LOAD obj/o_kougeki017.o
LOAD obj/o_kougeki018.o
LOAD obj/o_kougeki019.o
LOAD obj/o_kougeki020.o
LOAD obj/o_yarare000.o
LOAD obj/o_yarare001.o
LOAD obj/o_yarare002.o
LOAD obj/o_yarare003.o
LOAD obj/o_yarare004.o
LOAD obj/o_yarare005.o
LOAD obj/o_yarare006.o
LOAD obj/o_yarare007.o
LOAD obj/o_yarare008.o
LOAD obj/o_yarare009.o
LOAD obj/o_yarare010.o
LOAD obj/o_yarare011.o
LOAD obj/o_yarare012.o
LOAD obj/o_yarare013.o
LOAD obj/o_yarare014.o
LOAD obj/o_yarare015.o
LOAD obj/o_yarare016.o
LOAD obj/o_yarare017.o
LOAD obj/o_yarare018.o
LOAD obj/o_yarare019.o
LOAD obj/o_yarare020.o
LOAD obj/o_fukiya000.o
LOAD obj/awa.o
LOAD obj/ring_32_64_left.o
LOAD obj/ring_32_64_right.o
LOAD bg_parts/umia_.o
LOAD bg_parts/umi_ab_256x512.o
LOAD bg_parts/sango1024x256.o
LOAD bg_parts/sora.o
LOAD bg_parts/light4.o
LOAD bg_parts/wave2nd1.o
LOAD bg_parts/wave2nd2.o
LOAD bg_parts/wave2nd3.o
LOAD C:/agb/lib//libagbsyscall.a
LOAD C:/agb/lib//libisagbprn.a
LOAD C:\PROGRA~1\CYGNUS\THUMBELF-000512\H-I686-CYGWIN32\BIN/../lib/gcc-lib/thumb-elf/2.9-arm-000512/libgcc.a
LOAD C:\PROGRA~1\CYGNUS\THUMBELF-000512\H-I686-CYGWIN32\BIN/../lib/gcc-lib/thumb-elf/2.9-arm-000512/../../../../thumb-elf/lib/libg.a
LOAD C:\PROGRA~1\CYGNUS\THUMBELF-000512\H-I686-CYGWIN32\BIN/../lib/gcc-lib/thumb-elf/2.9-arm-000512/../../../../thumb-elf/lib/libc.a
LOAD C:\PROGRA~1\CYGNUS\THUMBELF-000512\H-I686-CYGWIN32\BIN/../lib/gcc-lib/thumb-elf/2.9-arm-000512/libgcc.a
Address of section .text set to 0x8000000
Address of section .bss set to 0x3000000
                0x00008000                .=0x8000

.interp
 *(.interp)

.hash
 *(.hash)

.dynsym
 *(.dynsym)

.dynstr
 *(.dynstr)

.gnu.version
 *(.gnu.version)

.gnu.version_d
 *(.gnu.version_d)

.gnu.version_r
 *(.gnu.version_r)

.rel.text
 *(.rel.text)
 *(.rel.text.*)
 *(.rel.gnu.linkonce.t*)

.rela.text
 *(.rela.text)
 *(.rela.text.*)
 *(.rela.gnu.linkonce.t*)

.rel.data
 *(.rel.data)
 *(.rel.data.*)
 *(.rel.gnu.linkonce.d*)

.rela.data
 *(.rela.data)
 *(.rela.data.*)
 *(.rela.gnu.linkonce.d*)

.rel.rodata
 *(.rel.rodata)
 *(.rel.rodata.*)
 *(.rel.gnu.linkonce.r*)

.rela.rodata
 *(.rela.rodata)
 *(.rela.rodata.*)
 *(.rela.gnu.linkonce.r*)

.rel.got
 *(.rel.got)

.rela.got
 *(.rela.got)

.rel.ctors
 *(.rel.ctors)

.rela.ctors
 *(.rela.ctors)

.rel.dtors
 *(.rel.dtors)

.rela.dtors
 *(.rela.dtors)

.rel.init
 *(.rel.init)

.rela.init
 *(.rela.init)

.rel.fini
 *(.rel.fini)

.rela.fini
 *(.rela.fini)

.rel.bss
 *(.rel.bss)

.rela.bss
 *(.rela.bss)

.rel.plt
 *(.rel.plt)

.rela.plt
 *(.rela.plt)

.init
 *(.init)

.plt
 *(.plt)

.text           0x08000000     0x2e84
 *(.text)
 .text          0x08000000      0x1cc crt0.o
                0x08000000                _start
                0x080000c0                start_vector
                0x080000fc                intr_main
 .text          0x080001cc      0x374 main.o
                0x080003d0                IntrDammy
                0x080003cc                VCountIntr
                0x080002bc                VBlankIntr
                0x080004bc                GameMain
                0x08000370                HBlankIntr
                0x080003d4                KeyRead
                0x08000400                GameInit
                0x080004e8                GameOver
                0x080001cc                AgbMain
 .text          0x08000540      0xd08 player.o
                0x08000cb0                Action3
                0x08000f80                Player_attack_anm
                0x08000ffc                Player_head_attack_anm
                0x08000ccc                PlayerAnim
                0x08000644                DrawPlayer
                0x08000540                InitPlayer
                0x08001050                Ajust_Light_Reflection
                0x08000d50                Player_kihon_idle_anm
                0x080010bc                InitPlayer_Awa
                0x08000f10                Player_idle_anm
                0x08001110                CreatePlayer_Awa
                0x08000ab0                ChangeWaterSpeed
                0x080011b8                DrawPlayer_Awa
                0x08000cec                Player_kihon_anm
                0x08000db4                Player_updown_anm
                0x08000ff8                Player_move_rl_anm
                0x0800099c                MovePlayer
                0x080010b8                BlinkPlayer
                0x080010e0                Player_AwaProc
                0x08000cb4                InitPlayerAnim
                0x080008b4                PlayerActionControl
                0x08000b60                Action1
                0x08001158                Player_AwaMove
                0x08000ea0                Player_jump_anm
                0x080005f0                PlayerProc
                0x08000914                Chang_Dir
                0x080007e4                RestrictPlayerPosition
                0x08000c0c                JumpPlayer
 .text          0x08001248      0x964 enemy.o
                0x080017f4                DrawEnemy
                0x080014a4                DeadCheckEnemy
                0x08001634                ShellAnim
                0x080018bc                InitAwa
                0x080018f8                AwaProc
                0x080018ac                EraseEnemy
                0x0800199c                DrawAwa
                0x08001928                CreateAwa
                0x080017f0                ShellDeadAnim
                0x08001410                HitCheck_Enemy
                0x08001448                HitEnemy
                0x08001a38                InitFukiya
                0x080015e8                LcdCheckEnemy
                0x08001248                InitEnemy
                0x08001668                ShellBaseAnim
                0x08001584                DeadMove
                0x08001540                MoveShell1
                0x08001a74                FukiyaProc
                0x08001508                ControlEnemyMove
                0x08001784                ShellDamageAnim
                0x08001580                ShellAttackMove
                0x080016f4                ShellAttackAnim
                0x08001308                EnemyProc
                0x08001af4                FukiyaMove
                0x08001368                CreateTeki
                0x08001aa4                CreateFukiya
                0x08001960                AwaMove
                0x0800157c                MoveShell2
                0x08001b0c                DrawFukiya
 .text          0x08001bac      0xbf8 bg.o
                0x0800268c                DeleteOceanB
                0x08002190                CoralRight
                0x080022ac                DrawLight
                0x08001e34                Init_Sky_ScreenDat
                0x080023d8                OceanA_Idle
                0x080024a0                DeleteOceanA
                0x08001bc4                Anm_wave2nd
                0x08001eec                DeleteSky
                0x08002444                DrawOceanA
                0x08001c98                Change_Bg_VRAM
                0x08002210                CoralLeft
                0x08001f40                SoraRight
                0x08002314                DeleteLight
                0x08001c74                BgProc
                0x0800239c                InitOceanAScreenDat
                0x080026a8                OceanB_Up
                0x080022a8                InitLightScreenDat
                0x080025cc                InitOceanB
                0x08002604                InitOceanBScreenDat
                0x08002080                InitCoralScreenDat
                0x08002294                CoralUpDown
                0x08001fc0                SoraLeft
                0x08002044                InitCoral
                0x08001c14                InitBg
                0x08001bac                initwave2nd
                0x080020c0                DrawCoral
                0x08002298                InitLight
                0x08002558                OceanA_Down
                0x08001ce8                UpdateBg
                0x08002364                InitOceanA
                0x08002724                OceanB_Down
                0x08002640                DrawOceanB
                0x08001e74                DrawSky
                0x080024e4                OceanA_Up
                0x08001dfc                InitSky
                0x0800213c                DeleteCoral
 .text          0x080027a4      0x34c hitcheck.o
                0x080028c4                Ring2Dolphin
                0x08002a18                RingPass
                0x080027a4                Fukiya2Dolphin
                0x080027fc                Dolphin2Enemy
 .text          0x08002af0      0x2c0 ring.o
                0x08002dac                RingHit
                0x08002af0                InitRing
                0x08002c38                DrawRing
                0x08002d70                RingPassed
                0x08002d44                RingNormal
                0x08002c00                CreateRing
                0x08002b60                RingProc
                0x08002bcc                RingStateControl
 .text          0x08002db0       0x3c C:\PROGRA~1\CYGNUS\THUMBELF-000512\H-I686-CYGWIN32\BIN/../lib/gcc-lib/thumb-elf/2.9-arm-000512/libgcc.a(_call_via_rX.o)
                0x08002db8                _call_via_r2
                0x08002dc8                _call_via_r6
                0x08002dc4                _call_via_r5
                0x08002dbc                _call_via_r3
                0x08002ddc                _call_via_fp
                0x08002dd0                _call_via_r8
                0x08002dcc                _call_via_r7
                0x08002db0                _call_via_r0
                0x08002dd8                _call_via_sl
                0x08002de4                _call_via_sp
                0x08002dd4                _call_via_r9
                0x08002dc0                _call_via_r4
                0x08002db4                _call_via_r1
                0x08002de0                _call_via_ip
                0x08002de8                _call_via_lr
 .text          0x08002dec       0x94 C:\PROGRA~1\CYGNUS\THUMBELF-000512\H-I686-CYGWIN32\BIN/../lib/gcc-lib/thumb-elf/2.9-arm-000512/libgcc.a(_divsi3.o)
                0x08002dec                __divsi3
 .text          0x08002e80        0x4 C:\PROGRA~1\CYGNUS\THUMBELF-000512\H-I686-CYGWIN32\BIN/../lib/gcc-lib/thumb-elf/2.9-arm-000512/libgcc.a(_dvmd_tls.o)
                0x08002e80                __div0
 *(.text.*)
 *(.stub)
 *(.gnu.warning)
 *(.gnu.linkonce.t*)
 *(.glue_7t)
 *(.glue_7)
                0x08002e84                _etext=.
                0x08002e84                PROVIDE (etext, .)

.fini
 *(.fini)

.rodata         0x08002e84    0x743c4
 *(.rodata)
 .rodata        0x08002e84       0x3c main.o
                0x08002e84                IntrTable
 .rodata        0x08002ec0       0x30 enemy.o
                0x08002ec0                Oam_def
                0x08002ed8                Oam_8x8dot
                0x08002ed0                Oam_16x16dot
                0x08002ec8                Oam_32x32dot
 .rodata        0x08002ef0       0x10 game_dat.o
                0x08002ef8                OamData_Sample
                0x08002ef0                Oam_16x8dot
 .rodata        0x08002f00        0x8 ring.o
                0x08002f00                Oam_32x64dot
 .rodata        0x08002f08     0x1200 obj/r_kihon0.o
                0x08003108                r_kihon0_Char
                0x08002f08                r_kihon0_Palette
 .rodata        0x08004108     0x1200 obj/r_kihon1.o
                0x08004308                r_kihon1_Char
                0x08004108                r_kihon1_Palette
 .rodata        0x08005308     0x1200 obj/r_kihon2.o
                0x08005308                r_kihon2_Palette
                0x08005508                r_kihon2_Char
 .rodata        0x08006508     0x1200 obj/r_kihon3.o
                0x08006708                r_kihon3_Char
                0x08006508                r_kihon3_Palette
 .rodata        0x08007708     0x1200 obj/r_kihon4.o
                0x08007708                r_kihon4_Palette
                0x08007908                r_kihon4_Char
 .rodata        0x08008908     0x1200 obj/r_kihon5.o
                0x08008b08                r_kihon5_Char
                0x08008908                r_kihon5_Palette
 .rodata        0x08009b08     0x1200 obj/r_kihon6.o
                0x08009b08                r_kihon6_Palette
                0x08009d08                r_kihon6_Char
 .rodata        0x0800ad08     0x1200 obj/r_kihon7.o
                0x0800af08                r_kihon7_Char
                0x0800ad08                r_kihon7_Palette
 .rodata        0x0800bf08     0x1200 obj/r_up0.o
                0x0800c108                r_up0_Char
                0x0800bf08                r_up0_Palette
 .rodata        0x0800d108     0x1200 obj/r_up1.o
                0x0800d308                r_up1_Char
                0x0800d108                r_up1_Palette
 .rodata        0x0800e308     0x1200 obj/r_up2.o
                0x0800e308                r_up2_Palette
                0x0800e508                r_up2_Char
 .rodata        0x0800f508     0x1200 obj/r_up3.o
                0x0800f508                r_up3_Palette
                0x0800f708                r_up3_Char
 .rodata        0x08010708     0x1200 obj/r_up4.o
                0x08010708                r_up4_Palette
                0x08010908                r_up4_Char
 .rodata        0x08011908     0x1200 obj/r_up5.o
                0x08011908                r_up5_Palette
                0x08011b08                r_up5_Char
 .rodata        0x08012b08     0x1200 obj/r_up6.o
                0x08012d08                r_up6_Char
                0x08012b08                r_up6_Palette
 .rodata        0x08013d08     0x1200 obj/r_up7.o
                0x08013d08                r_up7_Palette
                0x08013f08                r_up7_Char
 .rodata        0x08014f08     0x1200 obj/r_up8.o
                0x08015108                r_up8_Char
                0x08014f08                r_up8_Palette
 .rodata        0x08016108     0x1200 obj/r_go_up0.o
                0x08016308                r_go_up0_Char
                0x08016108                r_go_up0_Palette
 .rodata        0x08017308     0x1200 obj/r_go_up1.o
                0x08017308                r_go_up1_Palette
                0x08017508                r_go_up1_Char
 .rodata        0x08018508     0x1200 obj/r_go_up2.o
                0x08018508                r_go_up2_Palette
                0x08018708                r_go_up2_Char
 .rodata        0x08019708     0x1200 obj/r_go_up3.o
                0x08019908                r_go_up3_Char
                0x08019708                r_go_up3_Palette
 .rodata        0x0801a908     0x1200 obj/r_go_up4.o
                0x0801a908                r_go_up4_Palette
                0x0801ab08                r_go_up4_Char
 .rodata        0x0801bb08     0x1200 obj/r_go_up5.o
                0x0801bd08                r_go_up5_Char
                0x0801bb08                r_go_up5_Palette
 .rodata        0x0801cd08     0x1200 obj/r_go_up6.o
                0x0801cf08                r_go_up6_Char
                0x0801cd08                r_go_up6_Palette
 .rodata        0x0801df08     0x1200 obj/r_go_up7.o
                0x0801e108                r_go_up7_Char
                0x0801df08                r_go_up7_Palette
 .rodata        0x0801f108     0x1200 obj/r_down0.o
                0x0801f308                r_down0_Char
                0x0801f108                r_down0_Palette
 .rodata        0x08020308     0x1200 obj/r_down1.o
                0x08020308                r_down1_Palette
                0x08020508                r_down1_Char
 .rodata        0x08021508     0x1200 obj/r_down2.o
                0x08021508                r_down2_Palette
                0x08021708                r_down2_Char
 .rodata        0x08022708     0x1200 obj/r_down3.o
                0x08022708                r_down3_Palette
                0x08022908                r_down3_Char
 .rodata        0x08023908     0x1200 obj/r_down4.o
                0x08023908                r_down4_Palette
                0x08023b08                r_down4_Char
 .rodata        0x08024b08     0x1200 obj/r_down5.o
                0x08024b08                r_down5_Palette
                0x08024d08                r_down5_Char
 .rodata        0x08025d08     0x1200 obj/r_down6.o
                0x08025d08                r_down6_Palette
                0x08025f08                r_down6_Char
 .rodata        0x08026f08     0x1200 obj/r_down7.o
                0x08026f08                r_down7_Palette
                0x08027108                r_down7_Char
 .rodata        0x08028108     0x1200 obj/r_down8.o
                0x08028108                r_down8_Palette
                0x08028308                r_down8_Char
 .rodata        0x08029308     0x1200 obj/r_go_down0.o
                0x08029508                r_go_down0_Char
                0x08029308                r_go_down0_Palette
 .rodata        0x0802a508     0x1200 obj/r_go_down1.o
                0x0802a708                r_go_down1_Char
                0x0802a508                r_go_down1_Palette
 .rodata        0x0802b708     0x1200 obj/r_go_down2.o
                0x0802b708                r_go_down2_Palette
                0x0802b908                r_go_down2_Char
 .rodata        0x0802c908     0x1200 obj/r_go_down3.o
                0x0802c908                r_go_down3_Palette
                0x0802cb08                r_go_down3_Char
 .rodata        0x0802db08     0x1200 obj/r_go_down4.o
                0x0802db08                r_go_down4_Palette
                0x0802dd08                r_go_down4_Char
 .rodata        0x0802ed08     0x1200 obj/r_go_down5.o
                0x0802ed08                r_go_down5_Palette
                0x0802ef08                r_go_down5_Char
 .rodata        0x0802ff08     0x1200 obj/r_go_down6.o
                0x08030108                r_go_down6_Char
                0x0802ff08                r_go_down6_Palette
 .rodata        0x08031108     0x1200 obj/r_go_down7.o
                0x08031108                r_go_down7_Palette
                0x08031308                r_go_down7_Char
 .rodata        0x08032308     0x1200 obj/r_jump0.o
                0x08032308                r_jump0_Palette
                0x08032508                r_jump0_Char
 .rodata        0x08033508     0x1200 obj/r_jump1.o
                0x08033708                r_jump1_Char
                0x08033508                r_jump1_Palette
 .rodata        0x08034708     0x1200 obj/r_jump2.o
                0x08034708                r_jump2_Palette
                0x08034908                r_jump2_Char
 .rodata        0x08035908     0x1200 obj/r_jump3.o
                0x08035b08                r_jump3_Char
                0x08035908                r_jump3_Palette
 .rodata        0x08036b08     0x1200 obj/r_jump4.o
                0x08036d08                r_jump4_Char
                0x08036b08                r_jump4_Palette
 .rodata        0x08037d08     0x1200 obj/r_jump5.o
                0x08037f08                r_jump5_Char
                0x08037d08                r_jump5_Palette
 .rodata        0x08038f08     0x1200 obj/r_jump6.o
                0x08038f08                r_jump6_Palette
                0x08039108                r_jump6_Char
 .rodata        0x0803a108     0x1200 obj/r_jump7.o
                0x0803a308                r_jump7_Char
                0x0803a108                r_jump7_Palette
 .rodata        0x0803b308     0x1200 obj/r_jump8.o
                0x0803b508                r_jump8_Char
                0x0803b308                r_jump8_Palette
 .rodata        0x0803c508     0x1200 obj/r_jump9.o
                0x0803c708                r_jump9_Char
                0x0803c508                r_jump9_Palette
 .rodata        0x0803d708     0x1200 obj/r_jump10.o
                0x0803d908                r_jump10_Char
                0x0803d708                r_jump10_Palette
 .rodata        0x0803e908     0x1200 obj/r_attack1.o
                0x0803eb08                r_attack1_Char
                0x0803e908                r_attack1_Palette
 .rodata        0x0803fb08     0x1200 obj/r_attack2.o
                0x0803fb08                r_attack2_Palette
                0x0803fd08                r_attack2_Char
 .rodata        0x08040d08     0x1200 obj/r_attack3.o
                0x08040d08                r_attack3_Palette
                0x08040f08                r_attack3_Char
 .rodata        0x08041f08     0x1200 obj/r_attack4.o
                0x08042108                r_attack4_Char
                0x08041f08                r_attack4_Palette
 .rodata        0x08043108     0x1200 obj/r_attack5.o
                0x08043108                r_attack5_Palette
                0x08043308                r_attack5_Char
 .rodata        0x08044308     0x1200 obj/r_attack6.o
                0x08044308                r_attack6_Palette
                0x08044508                r_attack6_Char
 .rodata        0x08045508     0x1200 obj/r_attack7.o
                0x08045708                r_attack7_Char
                0x08045508                r_attack7_Palette
 .rodata        0x08046708      0x600 obj/o_kihon001.o
                0x08046908                o_kihon001_Char
                0x08046708                o_kihon001_Palette
 .rodata        0x08046d08      0x600 obj/o_kihon002.o
                0x08046d08                o_kihon002_Palette
                0x08046f08                o_kihon002_Char
 .rodata        0x08047308      0x600 obj/o_kihon003.o
                0x08047308                o_kihon003_Palette
                0x08047508                o_kihon003_Char
 .rodata        0x08047908      0x600 obj/o_kihon004.o
                0x08047908                o_kihon004_Palette
                0x08047b08                o_kihon004_Char
 .rodata        0x08047f08      0x600 obj/o_kihon005.o
                0x08048108                o_kihon005_Char
                0x08047f08                o_kihon005_Palette
 .rodata        0x08048508      0x600 obj/o_kihon006.o
                0x08048508                o_kihon006_Palette
                0x08048708                o_kihon006_Char
 .rodata        0x08048b08      0x600 obj/o_kihon007.o
                0x08048b08                o_kihon007_Palette
                0x08048d08                o_kihon007_Char
 .rodata        0x08049108      0x600 obj/o_kihon008.o
                0x08049308                o_kihon008_Char
                0x08049108                o_kihon008_Palette
 .rodata        0x08049708      0x600 obj/o_kihon009.o
                0x08049708                o_kihon009_Palette
                0x08049908                o_kihon009_Char
 .rodata        0x08049d08      0x600 obj/o_kihon010.o
                0x08049f08                o_kihon010_Char
                0x08049d08                o_kihon010_Palette
 .rodata        0x0804a308      0x600 obj/o_kougeki000.o
                0x0804a508                o_kougeki000_Char
                0x0804a308                o_kougeki000_Palette
 .rodata        0x0804a908      0x600 obj/o_kougeki001.o
                0x0804ab08                o_kougeki001_Char
                0x0804a908                o_kougeki001_Palette
 .rodata        0x0804af08      0x600 obj/o_kougeki002.o
                0x0804af08                o_kougeki002_Palette
                0x0804b108                o_kougeki002_Char
 .rodata        0x0804b508      0x600 obj/o_kougeki003.o
                0x0804b508                o_kougeki003_Palette
                0x0804b708                o_kougeki003_Char
 .rodata        0x0804bb08      0x600 obj/o_kougeki004.o
                0x0804bb08                o_kougeki004_Palette
                0x0804bd08                o_kougeki004_Char
 .rodata        0x0804c108      0x600 obj/o_kougeki005.o
                0x0804c308                o_kougeki005_Char
                0x0804c108                o_kougeki005_Palette
 .rodata        0x0804c708      0x600 obj/o_kougeki006.o
                0x0804c708                o_kougeki006_Palette
                0x0804c908                o_kougeki006_Char
 .rodata        0x0804cd08      0x600 obj/o_kougeki007.o
                0x0804cd08                o_kougeki007_Palette
                0x0804cf08                o_kougeki007_Char
 .rodata        0x0804d308      0x600 obj/o_kougeki008.o
                0x0804d308                o_kougeki008_Palette
                0x0804d508                o_kougeki008_Char
 .rodata        0x0804d908      0x600 obj/o_kougeki009.o
                0x0804db08                o_kougeki009_Char
                0x0804d908                o_kougeki009_Palette
 .rodata        0x0804df08      0x600 obj/o_kougeki010.o
                0x0804e108                o_kougeki010_Char
                0x0804df08                o_kougeki010_Palette
 .rodata        0x0804e508      0x600 obj/o_kougeki011.o
                0x0804e708                o_kougeki011_Char
                0x0804e508                o_kougeki011_Palette
 .rodata        0x0804eb08      0x600 obj/o_kougeki012.o
                0x0804eb08                o_kougeki012_Palette
                0x0804ed08                o_kougeki012_Char
 .rodata        0x0804f108      0x600 obj/o_kougeki013.o
                0x0804f308                o_kougeki013_Char
                0x0804f108                o_kougeki013_Palette
 .rodata        0x0804f708      0x600 obj/o_kougeki014.o
                0x0804f708                o_kougeki014_Palette
                0x0804f908                o_kougeki014_Char
 .rodata        0x0804fd08      0x600 obj/o_kougeki015.o
                0x0804ff08                o_kougeki015_Char
                0x0804fd08                o_kougeki015_Palette
 .rodata        0x08050308      0x600 obj/o_kougeki016.o
                0x08050308                o_kougeki016_Palette
                0x08050508                o_kougeki016_Char
 .rodata        0x08050908      0x600 obj/o_kougeki017.o
                0x08050b08                o_kougeki017_Char
                0x08050908                o_kougeki017_Palette
 .rodata        0x08050f08      0x600 obj/o_kougeki018.o
                0x08051108                o_kougeki018_Char
                0x08050f08                o_kougeki018_Palette
 .rodata        0x08051508      0x600 obj/o_kougeki019.o
                0x08051708                o_kougeki019_Char
                0x08051508                o_kougeki019_Palette
 .rodata        0x08051b08      0x600 obj/o_kougeki020.o
                0x08051d08                o_kougeki020_Char
                0x08051b08                o_kougeki020_Palette
 .rodata        0x08052108      0x600 obj/o_yarare000.o
                0x08052308                o_yarare000_Char
                0x08052108                o_yarare000_Palette
 .rodata        0x08052708      0x600 obj/o_yarare001.o
                0x08052908                o_yarare001_Char
                0x08052708                o_yarare001_Palette
 .rodata        0x08052d08      0x600 obj/o_yarare002.o
                0x08052d08                o_yarare002_Palette
                0x08052f08                o_yarare002_Char
 .rodata        0x08053308      0x600 obj/o_yarare003.o
                0x08053508                o_yarare003_Char
                0x08053308                o_yarare003_Palette
 .rodata        0x08053908      0x600 obj/o_yarare004.o
                0x08053908                o_yarare004_Palette
                0x08053b08                o_yarare004_Char
 .rodata        0x08053f08      0x600 obj/o_yarare005.o
                0x08054108                o_yarare005_Char
                0x08053f08                o_yarare005_Palette
 .rodata        0x08054508      0x600 obj/o_yarare006.o
                0x08054708                o_yarare006_Char
                0x08054508                o_yarare006_Palette
 .rodata        0x08054b08      0x600 obj/o_yarare007.o
                0x08054d08                o_yarare007_Char
                0x08054b08                o_yarare007_Palette
 .rodata        0x08055108      0x600 obj/o_yarare008.o
                0x08055108                o_yarare008_Palette
                0x08055308                o_yarare008_Char
 .rodata        0x08055708      0x600 obj/o_yarare009.o
                0x08055708                o_yarare009_Palette
                0x08055908                o_yarare009_Char
 .rodata        0x08055d08      0x600 obj/o_yarare010.o
                0x08055f08                o_yarare010_Char
                0x08055d08                o_yarare010_Palette
 .rodata        0x08056308      0x600 obj/o_yarare011.o
                0x08056508                o_yarare011_Char
                0x08056308                o_yarare011_Palette
 .rodata        0x08056908      0x600 obj/o_yarare012.o
                0x08056b08                o_yarare012_Char
                0x08056908                o_yarare012_Palette
 .rodata        0x08056f08      0x600 obj/o_yarare013.o
                0x08056f08                o_yarare013_Palette
                0x08057108                o_yarare013_Char
 .rodata        0x08057508      0x600 obj/o_yarare014.o
                0x08057508                o_yarare014_Palette
                0x08057708                o_yarare014_Char
 .rodata        0x08057b08      0x600 obj/o_yarare015.o
                0x08057d08                o_yarare015_Char
                0x08057b08                o_yarare015_Palette
 .rodata        0x08058108      0x600 obj/o_yarare016.o
                0x08058108                o_yarare016_Palette
                0x08058308                o_yarare016_Char
 .rodata        0x08058708      0x600 obj/o_yarare017.o
                0x08058708                o_yarare017_Palette
                0x08058908                o_yarare017_Char
 .rodata        0x08058d08      0x600 obj/o_yarare018.o
                0x08058f08                o_yarare018_Char
                0x08058d08                o_yarare018_Palette
 .rodata        0x08059308      0x600 obj/o_yarare019.o
                0x08059308                o_yarare019_Palette
                0x08059508                o_yarare019_Char
 .rodata        0x08059908      0x600 obj/o_yarare020.o
                0x08059908                o_yarare020_Palette
                0x08059b08                o_yarare020_Char
 .rodata        0x08059f08      0x280 obj/o_fukiya000.o
                0x08059f08                o_fukiya000_Palette
                0x0805a108                o_fukiya000_Char
 .rodata        0x0805a188      0x240 obj/awa.o
                0x0805a388                awa_Char
                0x0805a188                awa_Palette
 .rodata        0x0805a3c8      0xa00 obj/ring_32_64_left.o
                0x0805a3c8                ring_32_64_left_Palette
                0x0805a5c8                ring_32_64_left_Char
 .rodata        0x0805adc8      0xa00 obj/ring_32_64_right.o
                0x0805adc8                ring_32_64_right_Palette
                0x0805afc8                ring_32_64_right_Char
 .rodata        0x0805b7c8     0x1680 bg_parts/umia_.o
                0x0805be48                umia__Map
                0x0805b7c8                umia__Palette
                0x0805b9c8                umia__Character
 .rodata        0x0805ce48     0x7f80 bg_parts/umi_ab_256x512.o
                0x0805ce48                umi_ab_256x512_Palette
                0x08063dc8                umi_ab_256x512_Map
                0x0805d048                umi_ab_256x512_Character
 .rodata        0x08064dc8     0x5fc0 bg_parts/sango1024x256.o
                0x08064dc8                sango1024x256_Palette
                0x08064fc8                sango1024x256_Character
                0x08068d88                sango1024x256_Map
 .rodata        0x0806ad88     0x8c00 bg_parts/sora.o
                0x08072988                sora_Map
                0x0806af88                sora_Character
                0x0806ad88                sora_Palette
 .rodata        0x08073988     0x2fc0 bg_parts/light4.o
                0x08076148                light4_Map
                0x08073988                light4_Palette
                0x08073b88                light4_Character
 .rodata        0x08076948      0x300 bg_parts/wave2nd1.o
                0x08076b48                wave2nd1_Char
                0x08076948                wave2nd1_Palette
 .rodata        0x08076c48      0x300 bg_parts/wave2nd2.o
                0x08076e48                wave2nd2_Char
                0x08076c48                wave2nd2_Palette
 .rodata        0x08076f48      0x300 bg_parts/wave2nd3.o
                0x08076f48                wave2nd3_Palette
                0x08077148                wave2nd3_Char
 *(.rodata.*)
 *(.gnu.linkonce.r*)

.rodata1
 *(.rodata1)
                0x08077348                .=(ALIGN(0x100)+(.&0xff))

.data           0x08077348      0xf5c
 *(.data)
 .data          0x08077348       0x38 main.o
 .data          0x08077380       0x5c player.o
 .data          0x080773dc      0x3c4 player_dat.o
                0x08077560                rick_normal_move_pat
                0x0807747c                r_down_pixel_tbl
                0x08077464                r_attack_pixel_tbl
                0x08077444                r_kihon_idle_pixel_tbl
                0x080776f8                rick_attack_pat
                0x080775b4                rick_kihon_idle_pat
                0x08077614                rick_jump_anm_pat
                0x0807742c                r_kihon_pixel_tbl
                0x08077710                rick_kihon_fast_pat
                0x080774a0                r_up_down_pixel_tbl
                0x08077514                r_jump_pixel_tbl
                0x0807773c                rick_jump_pat
 .data          0x080777a0       0x5c enemy.o
                0x080777f0                anm_state
 .data          0x080777fc      0x3c0 enemy_dat.o
                0x08077980                shell_yarare_pix_tbl
                0x08077b6c                enemy_Oam_Data
                0x080779d4                shell_yarare_anm_pat
                0x080778c4                shell_attack_pix_tbl
                0x0807784c                shell_base_pix_tbl
                0x08077a7c                shell_map_dat
                0x08077874                shell_base_anm_pat
                0x08077918                shell_attack_anm_pat
 .data          0x08077bbc      0x500 game_dat.o
                0x08077dbc                cos_tbl
                0x08077bbc                sin_tbl
                0x08077fbc                sintable
 .data          0x080780bc       0x60 bg.o
                0x080780ec                wave2nd_pat
 .data          0x0807811c       0x5c hitcheck.o
 .data          0x08078178      0x12c ring.o
                0x080781b4                ring_map_dat
 *(.data.*)
 *(.gnu.linkonce.d*)

.data1
 *(.data1)

.ctors
 EXCLUDE_FILE ( *crtend.o )*(.ctors)
 *(SORT(.ctors.*))
 *crtend(.ctors)

.dtors
 EXCLUDE_FILE ( *crtend.o )*(.dtors)
 *(SORT(.dtors.*))
 *crtend.o(.dtors)

.got
 *(.got.plt)
 *(.got)

.dynamic
 *(.dynamic)

.sdata
 *(.sdata)
 *(.sdata.*)
                0x080782a4                _edata=.
                0x080782a4                PROVIDE (edata, .)
                0x080782a4                __bss_start=.
                0x080782a4                __bss_start__=.

.sbss
 *(.sbss)
 *(.scommon)

.bss            0x03000000     0x36b0
 *(.dynbss)
 *(.bss)
 *(.bss.*)
 *(COMMON)
 COMMON         0x03000000      0xdac main.o
                                  0x0 (size before relaxing)
                0x03000000                Oam
                0x03000480                hz
                0x03000484                v_phase
                0x03000488                Cont
                0x0300048c                state
                0x03000490                rasttable
                0x03000590                Trg
                0x03000594                counter
                0x030005a0                IntrMainBuf
                0x03000da0                amp_r
                0x03000da4                IntrCheck
                0x03000da8                offset
 *fill*         0x03000dac        0x4
 COMMON         0x03000db0       0xb0 player.o
                                  0x0 (size before relaxing)
                0x03000db0                player
                0x03000e00                player_awa
 COMMON         0x03000e60      0x478 enemy.o
                                  0x0 (size before relaxing)
                0x03000e60                fukiya
                0x03000ea0                awa
                0x03000fe0                dEnemy
 *fill*         0x030012d8        0x8
 COMMON         0x030012e0     0x2150 bg.o
                                  0x0 (size before relaxing)
                0x030012e0                Sky
                0x03001314                DisplayArea
                0x03001320                Light
                0x03001360                wave2nd
                0x03001370                OceanA
                0x030013a4                sora_xPos
                0x030013b0                Sango_ScreenDat
                0x03001bb0                UmiA_ScreenDat
                0x030023b0                Bg2_ScreenDat
                0x03002bb0                Coral
                0x03002bf0                OceanB
                0x03002c24                ocean_xPos
                0x03002c30                Sky_ScreenDat
 COMMON         0x03003430      0x280 ring.o
                                  0x0 (size before relaxing)
                0x03003430                ring
                0x030036b0                .=ALIGN(0x4)
                0x030036b0                .=ALIGN(0x4)
                0x030036b0                _end=.
                0x030036b0                _bss_end__=.
                0x030036b0                __bss_end__=.
                0x030036b0                PROVIDE (end, .)

.stab
 *(.stab)

.stabstr
 *(.stabstr)

.stab.excl
 *(.stab.excl)

.stab.exclstr
 *(.stab.exclstr)

.stab.index
 *(.stab.index)

.stab.indexstr
 *(.stab.indexstr)

.comment
 *(.comment)

.debug
 *(.debug)

.line
 *(.line)

.debug_srcinfo
 *(.debug_srcinfo)

.debug_sfnames
 *(.debug_sfnames)

.debug_aranges  0x00000000       0xc0
 *(.debug_aranges)
 .debug_aranges
                0x00000000       0x20 main.o
 .debug_aranges
                0x00000020       0x20 player.o
 .debug_aranges
                0x00000040       0x20 enemy.o
 .debug_aranges
                0x00000060       0x20 bg.o
 .debug_aranges
                0x00000080       0x20 hitcheck.o
 .debug_aranges
                0x000000a0       0x20 ring.o

.debug_pubnames
                0x00000000     0x294e
 *(.debug_pubnames)
 .debug_pubnames
                0x00000000      0x11d main.o
 .debug_pubnames
                0x0000011d      0x248 player.o
 .debug_pubnames
                0x00000365      0x121 player_dat.o
 .debug_pubnames
                0x00000486      0x241 enemy.o
 .debug_pubnames
                0x000006c7       0xc9 enemy_dat.o
 .debug_pubnames
                0x00000790       0x5a game_dat.o
 .debug_pubnames
                0x000007ea      0x313 bg.o
 .debug_pubnames
                0x00000afd       0x55 hitcheck.o
 .debug_pubnames
                0x00000b52       0xb2 ring.o
 .debug_pubnames
                0x00000c04       0x39 obj/r_kihon0.o
 .debug_pubnames
                0x00000c3d       0x39 obj/r_kihon1.o
 .debug_pubnames
                0x00000c76       0x39 obj/r_kihon2.o
 .debug_pubnames
                0x00000caf       0x39 obj/r_kihon3.o
 .debug_pubnames
                0x00000ce8       0x39 obj/r_kihon4.o
 .debug_pubnames
                0x00000d21       0x39 obj/r_kihon5.o
 .debug_pubnames
                0x00000d5a       0x39 obj/r_kihon6.o
 .debug_pubnames
                0x00000d93       0x39 obj/r_kihon7.o
 .debug_pubnames
                0x00000dcc       0x33 obj/r_up0.o
 .debug_pubnames
                0x00000dff       0x33 obj/r_up1.o
 .debug_pubnames
                0x00000e32       0x33 obj/r_up2.o
 .debug_pubnames
                0x00000e65       0x33 obj/r_up3.o
 .debug_pubnames
                0x00000e98       0x33 obj/r_up4.o
 .debug_pubnames
                0x00000ecb       0x33 obj/r_up5.o
 .debug_pubnames
                0x00000efe       0x33 obj/r_up6.o
 .debug_pubnames
                0x00000f31       0x33 obj/r_up7.o
 .debug_pubnames
                0x00000f64       0x33 obj/r_up8.o
 .debug_pubnames
                0x00000f97       0x39 obj/r_go_up0.o
 .debug_pubnames
                0x00000fd0       0x39 obj/r_go_up1.o
 .debug_pubnames
                0x00001009       0x39 obj/r_go_up2.o
 .debug_pubnames
                0x00001042       0x39 obj/r_go_up3.o
 .debug_pubnames
                0x0000107b       0x39 obj/r_go_up4.o
 .debug_pubnames
                0x000010b4       0x39 obj/r_go_up5.o
 .debug_pubnames
                0x000010ed       0x39 obj/r_go_up6.o
 .debug_pubnames
                0x00001126       0x39 obj/r_go_up7.o
 .debug_pubnames
                0x0000115f       0x37 obj/r_down0.o
 .debug_pubnames
                0x00001196       0x37 obj/r_down1.o
 .debug_pubnames
                0x000011cd       0x37 obj/r_down2.o
 .debug_pubnames
                0x00001204       0x37 obj/r_down3.o
 .debug_pubnames
                0x0000123b       0x37 obj/r_down4.o
 .debug_pubnames
                0x00001272       0x37 obj/r_down5.o
 .debug_pubnames
                0x000012a9       0x37 obj/r_down6.o
 .debug_pubnames
                0x000012e0       0x37 obj/r_down7.o
 .debug_pubnames
                0x00001317       0x37 obj/r_down8.o
 .debug_pubnames
                0x0000134e       0x3d obj/r_go_down0.o
 .debug_pubnames
                0x0000138b       0x3d obj/r_go_down1.o
 .debug_pubnames
                0x000013c8       0x3d obj/r_go_down2.o
 .debug_pubnames
                0x00001405       0x3d obj/r_go_down3.o
 .debug_pubnames
                0x00001442       0x3d obj/r_go_down4.o
 .debug_pubnames
                0x0000147f       0x3d obj/r_go_down5.o
 .debug_pubnames
                0x000014bc       0x3d obj/r_go_down6.o
 .debug_pubnames
                0x000014f9       0x3d obj/r_go_down7.o
 .debug_pubnames
                0x00001536       0x37 obj/r_jump0.o
 .debug_pubnames
                0x0000156d       0x37 obj/r_jump1.o
 .debug_pubnames
                0x000015a4       0x37 obj/r_jump2.o
 .debug_pubnames
                0x000015db       0x37 obj/r_jump3.o
 .debug_pubnames
                0x00001612       0x37 obj/r_jump4.o
 .debug_pubnames
                0x00001649       0x37 obj/r_jump5.o
 .debug_pubnames
                0x00001680       0x37 obj/r_jump6.o
 .debug_pubnames
                0x000016b7       0x37 obj/r_jump7.o
 .debug_pubnames
                0x000016ee       0x37 obj/r_jump8.o
 .debug_pubnames
                0x00001725       0x37 obj/r_jump9.o
 .debug_pubnames
                0x0000175c       0x39 obj/r_jump10.o
 .debug_pubnames
                0x00001795       0x3b obj/r_attack1.o
 .debug_pubnames
                0x000017d0       0x3b obj/r_attack2.o
 .debug_pubnames
                0x0000180b       0x3b obj/r_attack3.o
 .debug_pubnames
                0x00001846       0x3b obj/r_attack4.o
 .debug_pubnames
                0x00001881       0x3b obj/r_attack5.o
 .debug_pubnames
                0x000018bc       0x3b obj/r_attack6.o
 .debug_pubnames
                0x000018f7       0x3b obj/r_attack7.o
 .debug_pubnames
                0x00001932       0x3d obj/o_kihon001.o
 .debug_pubnames
                0x0000196f       0x3d obj/o_kihon002.o
 .debug_pubnames
                0x000019ac       0x3d obj/o_kihon003.o
 .debug_pubnames
                0x000019e9       0x3d obj/o_kihon004.o
 .debug_pubnames
                0x00001a26       0x3d obj/o_kihon005.o
 .debug_pubnames
                0x00001a63       0x3d obj/o_kihon006.o
 .debug_pubnames
                0x00001aa0       0x3d obj/o_kihon007.o
 .debug_pubnames
                0x00001add       0x3d obj/o_kihon008.o
 .debug_pubnames
                0x00001b1a       0x3d obj/o_kihon009.o
 .debug_pubnames
                0x00001b57       0x3d obj/o_kihon010.o
 .debug_pubnames
                0x00001b94       0x41 obj/o_kougeki000.o
 .debug_pubnames
                0x00001bd5       0x41 obj/o_kougeki001.o
 .debug_pubnames
                0x00001c16       0x41 obj/o_kougeki002.o
 .debug_pubnames
                0x00001c57       0x41 obj/o_kougeki003.o
 .debug_pubnames
                0x00001c98       0x41 obj/o_kougeki004.o
 .debug_pubnames
                0x00001cd9       0x41 obj/o_kougeki005.o
 .debug_pubnames
                0x00001d1a       0x41 obj/o_kougeki006.o
 .debug_pubnames
                0x00001d5b       0x41 obj/o_kougeki007.o
 .debug_pubnames
                0x00001d9c       0x41 obj/o_kougeki008.o
 .debug_pubnames
                0x00001ddd       0x41 obj/o_kougeki009.o
 .debug_pubnames
                0x00001e1e       0x41 obj/o_kougeki010.o
 .debug_pubnames
                0x00001e5f       0x41 obj/o_kougeki011.o
 .debug_pubnames
                0x00001ea0       0x41 obj/o_kougeki012.o
 .debug_pubnames
                0x00001ee1       0x41 obj/o_kougeki013.o
 .debug_pubnames
                0x00001f22       0x41 obj/o_kougeki014.o
 .debug_pubnames
                0x00001f63       0x41 obj/o_kougeki015.o
 .debug_pubnames
                0x00001fa4       0x41 obj/o_kougeki016.o
 .debug_pubnames
                0x00001fe5       0x41 obj/o_kougeki017.o
 .debug_pubnames
                0x00002026       0x41 obj/o_kougeki018.o
 .debug_pubnames
                0x00002067       0x41 obj/o_kougeki019.o
 .debug_pubnames
                0x000020a8       0x41 obj/o_kougeki020.o
 .debug_pubnames
                0x000020e9       0x3f obj/o_yarare000.o
 .debug_pubnames
                0x00002128       0x3f obj/o_yarare001.o
 .debug_pubnames
                0x00002167       0x3f obj/o_yarare002.o
 .debug_pubnames
                0x000021a6       0x3f obj/o_yarare003.o
 .debug_pubnames
                0x000021e5       0x3f obj/o_yarare004.o
 .debug_pubnames
                0x00002224       0x3f obj/o_yarare005.o
 .debug_pubnames
                0x00002263       0x3f obj/o_yarare006.o
 .debug_pubnames
                0x000022a2       0x3f obj/o_yarare007.o
 .debug_pubnames
                0x000022e1       0x3f obj/o_yarare008.o
 .debug_pubnames
                0x00002320       0x3f obj/o_yarare009.o
 .debug_pubnames
                0x0000235f       0x3f obj/o_yarare010.o
 .debug_pubnames
                0x0000239e       0x3f obj/o_yarare011.o
 .debug_pubnames
                0x000023dd       0x3f obj/o_yarare012.o
 .debug_pubnames
                0x0000241c       0x3f obj/o_yarare013.o
 .debug_pubnames
                0x0000245b       0x3f obj/o_yarare014.o
 .debug_pubnames
                0x0000249a       0x3f obj/o_yarare015.o
 .debug_pubnames
                0x000024d9       0x3f obj/o_yarare016.o
 .debug_pubnames
                0x00002518       0x3f obj/o_yarare017.o
 .debug_pubnames
                0x00002557       0x3f obj/o_yarare018.o
 .debug_pubnames
                0x00002596       0x3f obj/o_yarare019.o
 .debug_pubnames
                0x000025d5       0x3f obj/o_yarare020.o
 .debug_pubnames
                0x00002614       0x3f obj/o_fukiya000.o
 .debug_pubnames
                0x00002653       0x2f obj/awa.o
 .debug_pubnames
                0x00002682       0x47 obj/ring_32_64_left.o
 .debug_pubnames
                0x000026c9       0x49 obj/ring_32_64_right.o
 .debug_pubnames
                0x00002712       0x46 bg_parts/umia_.o
 .debug_pubnames
                0x00002758       0x61 bg_parts/umi_ab_256x512.o
 .debug_pubnames
                0x000027b9       0x5e bg_parts/sango1024x256.o
 .debug_pubnames
                0x00002817       0x43 bg_parts/sora.o
 .debug_pubnames
                0x0000285a       0x49 bg_parts/light4.o
 .debug_pubnames
                0x000028a3       0x39 bg_parts/wave2nd1.o
 .debug_pubnames
                0x000028dc       0x39 bg_parts/wave2nd2.o
 .debug_pubnames
                0x00002915       0x39 bg_parts/wave2nd3.o

.debug_info     0x00000000   0x152c67
 *(.debug_info)
 .debug_info    0x00000000     0x385b main.o
 .debug_info    0x0000385b     0x4493 player.o
 .debug_info    0x00007cee     0x3e1d player_dat.o
 .debug_info    0x0000bb0b     0x43b2 enemy.o
 .debug_info    0x0000febd     0x3eba enemy_dat.o
 .debug_info    0x00013d77     0x2e46 game_dat.o
 .debug_info    0x00016bbd     0x4296 bg.o
 .debug_info    0x0001ae53     0x3b5f hitcheck.o
 .debug_info    0x0001e9b2     0x3761 ring.o
 .debug_info    0x00022113     0x274b obj/r_kihon0.o
 .debug_info    0x0002485e     0x274b obj/r_kihon1.o
 .debug_info    0x00026fa9     0x274b obj/r_kihon2.o
 .debug_info    0x000296f4     0x274b obj/r_kihon3.o
 .debug_info    0x0002be3f     0x274b obj/r_kihon4.o
 .debug_info    0x0002e58a     0x274b obj/r_kihon5.o
 .debug_info    0x00030cd5     0x274b obj/r_kihon6.o
 .debug_info    0x00033420     0x274b obj/r_kihon7.o
 .debug_info    0x00035b6b     0x2742 obj/r_up0.o
 .debug_info    0x000382ad     0x2742 obj/r_up1.o
 .debug_info    0x0003a9ef     0x2742 obj/r_up2.o
 .debug_info    0x0003d131     0x2742 obj/r_up3.o
 .debug_info    0x0003f873     0x2742 obj/r_up4.o
 .debug_info    0x00041fb5     0x2742 obj/r_up5.o
 .debug_info    0x000446f7     0x2742 obj/r_up6.o
 .debug_info    0x00046e39     0x2742 obj/r_up7.o
 .debug_info    0x0004957b     0x2742 obj/r_up8.o
 .debug_info    0x0004bcbd     0x274b obj/r_go_up0.o
 .debug_info    0x0004e408     0x274b obj/r_go_up1.o
 .debug_info    0x00050b53     0x274b obj/r_go_up2.o
 .debug_info    0x0005329e     0x274b obj/r_go_up3.o
 .debug_info    0x000559e9     0x274b obj/r_go_up4.o
 .debug_info    0x00058134     0x274b obj/r_go_up5.o
 .debug_info    0x0005a87f     0x274b obj/r_go_up6.o
 .debug_info    0x0005cfca     0x274b obj/r_go_up7.o
 .debug_info    0x0005f715     0x2748 obj/r_down0.o
 .debug_info    0x00061e5d     0x2748 obj/r_down1.o
 .debug_info    0x000645a5     0x2748 obj/r_down2.o
 .debug_info    0x00066ced     0x2748 obj/r_down3.o
 .debug_info    0x00069435     0x2748 obj/r_down4.o
 .debug_info    0x0006bb7d     0x2748 obj/r_down5.o
 .debug_info    0x0006e2c5     0x2748 obj/r_down6.o
 .debug_info    0x00070a0d     0x2748 obj/r_down7.o
 .debug_info    0x00073155     0x2748 obj/r_down8.o
 .debug_info    0x0007589d     0x2751 obj/r_go_down0.o
 .debug_info    0x00077fee     0x2751 obj/r_go_down1.o
 .debug_info    0x0007a73f     0x2751 obj/r_go_down2.o
 .debug_info    0x0007ce90     0x2751 obj/r_go_down3.o
 .debug_info    0x0007f5e1     0x2751 obj/r_go_down4.o
 .debug_info    0x00081d32     0x2751 obj/r_go_down5.o
 .debug_info    0x00084483     0x2751 obj/r_go_down6.o
 .debug_info    0x00086bd4     0x2751 obj/r_go_down7.o
 .debug_info    0x00089325     0x2748 obj/r_jump0.o
 .debug_info    0x0008ba6d     0x2748 obj/r_jump1.o
 .debug_info    0x0008e1b5     0x2748 obj/r_jump2.o
 .debug_info    0x000908fd     0x2748 obj/r_jump3.o
 .debug_info    0x00093045     0x2748 obj/r_jump4.o
 .debug_info    0x0009578d     0x2748 obj/r_jump5.o
 .debug_info    0x00097ed5     0x2748 obj/r_jump6.o
 .debug_info    0x0009a61d     0x2748 obj/r_jump7.o
 .debug_info    0x0009cd65     0x2748 obj/r_jump8.o
 .debug_info    0x0009f4ad     0x2748 obj/r_jump9.o
 .debug_info    0x000a1bf5     0x274b obj/r_jump10.o
 .debug_info    0x000a4340     0x274e obj/r_attack1.o
 .debug_info    0x000a6a8e     0x274e obj/r_attack2.o
 .debug_info    0x000a91dc     0x274e obj/r_attack3.o
 .debug_info    0x000ab92a     0x274e obj/r_attack4.o
 .debug_info    0x000ae078     0x274e obj/r_attack5.o
 .debug_info    0x000b07c6     0x274e obj/r_attack6.o
 .debug_info    0x000b2f14     0x274e obj/r_attack7.o
 .debug_info    0x000b5662     0x2751 obj/o_kihon001.o
 .debug_info    0x000b7db3     0x2751 obj/o_kihon002.o
 .debug_info    0x000ba504     0x2751 obj/o_kihon003.o
 .debug_info    0x000bcc55     0x2751 obj/o_kihon004.o
 .debug_info    0x000bf3a6     0x2751 obj/o_kihon005.o
 .debug_info    0x000c1af7     0x2751 obj/o_kihon006.o
 .debug_info    0x000c4248     0x2751 obj/o_kihon007.o
 .debug_info    0x000c6999     0x2751 obj/o_kihon008.o
 .debug_info    0x000c90ea     0x2751 obj/o_kihon009.o
 .debug_info    0x000cb83b     0x2751 obj/o_kihon010.o
 .debug_info    0x000cdf8c     0x2757 obj/o_kougeki000.o
 .debug_info    0x000d06e3     0x2757 obj/o_kougeki001.o
 .debug_info    0x000d2e3a     0x2757 obj/o_kougeki002.o
 .debug_info    0x000d5591     0x2757 obj/o_kougeki003.o
 .debug_info    0x000d7ce8     0x2757 obj/o_kougeki004.o
 .debug_info    0x000da43f     0x2757 obj/o_kougeki005.o
 .debug_info    0x000dcb96     0x2757 obj/o_kougeki006.o
 .debug_info    0x000df2ed     0x2757 obj/o_kougeki007.o
 .debug_info    0x000e1a44     0x2757 obj/o_kougeki008.o
 .debug_info    0x000e419b     0x2757 obj/o_kougeki009.o
 .debug_info    0x000e68f2     0x2757 obj/o_kougeki010.o
 .debug_info    0x000e9049     0x2757 obj/o_kougeki011.o
 .debug_info    0x000eb7a0     0x2757 obj/o_kougeki012.o
 .debug_info    0x000edef7     0x2757 obj/o_kougeki013.o
 .debug_info    0x000f064e     0x2757 obj/o_kougeki014.o
 .debug_info    0x000f2da5     0x2757 obj/o_kougeki015.o
 .debug_info    0x000f54fc     0x2757 obj/o_kougeki016.o
 .debug_info    0x000f7c53     0x2757 obj/o_kougeki017.o
 .debug_info    0x000fa3aa     0x2757 obj/o_kougeki018.o
 .debug_info    0x000fcb01     0x2757 obj/o_kougeki019.o
 .debug_info    0x000ff258     0x2757 obj/o_kougeki020.o
 .debug_info    0x001019af     0x2754 obj/o_yarare000.o
 .debug_info    0x00104103     0x2754 obj/o_yarare001.o
 .debug_info    0x00106857     0x2754 obj/o_yarare002.o
 .debug_info    0x00108fab     0x2754 obj/o_yarare003.o
 .debug_info    0x0010b6ff     0x2754 obj/o_yarare004.o
 .debug_info    0x0010de53     0x2754 obj/o_yarare005.o
 .debug_info    0x001105a7     0x2754 obj/o_yarare006.o
 .debug_info    0x00112cfb     0x2754 obj/o_yarare007.o
 .debug_info    0x0011544f     0x2754 obj/o_yarare008.o
 .debug_info    0x00117ba3     0x2754 obj/o_yarare009.o
 .debug_info    0x0011a2f7     0x2754 obj/o_yarare010.o
 .debug_info    0x0011ca4b     0x2754 obj/o_yarare011.o
 .debug_info    0x0011f19f     0x2754 obj/o_yarare012.o
 .debug_info    0x001218f3     0x2754 obj/o_yarare013.o
 .debug_info    0x00124047     0x2754 obj/o_yarare014.o
 .debug_info    0x0012679b     0x2754 obj/o_yarare015.o
 .debug_info    0x00128eef     0x2754 obj/o_yarare016.o
 .debug_info    0x0012b643     0x2754 obj/o_yarare017.o
 .debug_info    0x0012dd97     0x2754 obj/o_yarare018.o
 .debug_info    0x001304eb     0x2754 obj/o_yarare019.o
 .debug_info    0x00132c3f     0x2754 obj/o_yarare020.o
 .debug_info    0x00135393     0x2753 obj/o_fukiya000.o
 .debug_info    0x00137ae6     0x273b obj/awa.o
 .debug_info    0x0013a221     0x2760 obj/ring_32_64_left.o
 .debug_info    0x0013c981     0x2763 obj/ring_32_64_right.o
 .debug_info    0x0013f0e4     0x2776 bg_parts/umia_.o
 .debug_info    0x0014185a     0x279b bg_parts/umi_ab_256x512.o
 .debug_info    0x00143ff5     0x2797 bg_parts/sango1024x256.o
 .debug_info    0x0014678c     0x2773 bg_parts/sora.o
 .debug_info    0x00148eff     0x277b bg_parts/light4.o
 .debug_info    0x0014b67a     0x274f bg_parts/wave2nd1.o
 .debug_info    0x0014ddc9     0x274f bg_parts/wave2nd2.o
 .debug_info    0x00150518     0x274f bg_parts/wave2nd3.o

.debug_abbrev   0x00000000     0x74ca
 *(.debug_abbrev)
 .debug_abbrev  0x00000000      0x1d8 main.o
 .debug_abbrev  0x000001d8      0x222 player.o
 .debug_abbrev  0x000003fa      0x173 player_dat.o
 .debug_abbrev  0x0000056d      0x203 enemy.o
 .debug_abbrev  0x00000770      0x162 enemy_dat.o
 .debug_abbrev  0x000008d2      0x101 game_dat.o
 .debug_abbrev  0x000009d3      0x212 bg.o
 .debug_abbrev  0x00000be5      0x19c hitcheck.o
 .debug_abbrev  0x00000d81      0x1ec ring.o
 .debug_abbrev  0x00000f6d       0xd1 obj/r_kihon0.o
 .debug_abbrev  0x0000103e       0xd1 obj/r_kihon1.o
 .debug_abbrev  0x0000110f       0xd1 obj/r_kihon2.o
 .debug_abbrev  0x000011e0       0xd1 obj/r_kihon3.o
 .debug_abbrev  0x000012b1       0xd1 obj/r_kihon4.o
 .debug_abbrev  0x00001382       0xd1 obj/r_kihon5.o
 .debug_abbrev  0x00001453       0xd1 obj/r_kihon6.o
 .debug_abbrev  0x00001524       0xd1 obj/r_kihon7.o
 .debug_abbrev  0x000015f5       0xd1 obj/r_up0.o
 .debug_abbrev  0x000016c6       0xd1 obj/r_up1.o
 .debug_abbrev  0x00001797       0xd1 obj/r_up2.o
 .debug_abbrev  0x00001868       0xd1 obj/r_up3.o
 .debug_abbrev  0x00001939       0xd1 obj/r_up4.o
 .debug_abbrev  0x00001a0a       0xd1 obj/r_up5.o
 .debug_abbrev  0x00001adb       0xd1 obj/r_up6.o
 .debug_abbrev  0x00001bac       0xd1 obj/r_up7.o
 .debug_abbrev  0x00001c7d       0xd1 obj/r_up8.o
 .debug_abbrev  0x00001d4e       0xd1 obj/r_go_up0.o
 .debug_abbrev  0x00001e1f       0xd1 obj/r_go_up1.o
 .debug_abbrev  0x00001ef0       0xd1 obj/r_go_up2.o
 .debug_abbrev  0x00001fc1       0xd1 obj/r_go_up3.o
 .debug_abbrev  0x00002092       0xd1 obj/r_go_up4.o
 .debug_abbrev  0x00002163       0xd1 obj/r_go_up5.o
 .debug_abbrev  0x00002234       0xd1 obj/r_go_up6.o
 .debug_abbrev  0x00002305       0xd1 obj/r_go_up7.o
 .debug_abbrev  0x000023d6       0xd1 obj/r_down0.o
 .debug_abbrev  0x000024a7       0xd1 obj/r_down1.o
 .debug_abbrev  0x00002578       0xd1 obj/r_down2.o
 .debug_abbrev  0x00002649       0xd1 obj/r_down3.o
 .debug_abbrev  0x0000271a       0xd1 obj/r_down4.o
 .debug_abbrev  0x000027eb       0xd1 obj/r_down5.o
 .debug_abbrev  0x000028bc       0xd1 obj/r_down6.o
 .debug_abbrev  0x0000298d       0xd1 obj/r_down7.o
 .debug_abbrev  0x00002a5e       0xd1 obj/r_down8.o
 .debug_abbrev  0x00002b2f       0xd1 obj/r_go_down0.o
 .debug_abbrev  0x00002c00       0xd1 obj/r_go_down1.o
 .debug_abbrev  0x00002cd1       0xd1 obj/r_go_down2.o
 .debug_abbrev  0x00002da2       0xd1 obj/r_go_down3.o
 .debug_abbrev  0x00002e73       0xd1 obj/r_go_down4.o
 .debug_abbrev  0x00002f44       0xd1 obj/r_go_down5.o
 .debug_abbrev  0x00003015       0xd1 obj/r_go_down6.o
 .debug_abbrev  0x000030e6       0xd1 obj/r_go_down7.o
 .debug_abbrev  0x000031b7       0xd1 obj/r_jump0.o
 .debug_abbrev  0x00003288       0xd1 obj/r_jump1.o
 .debug_abbrev  0x00003359       0xd1 obj/r_jump2.o
 .debug_abbrev  0x0000342a       0xd1 obj/r_jump3.o
 .debug_abbrev  0x000034fb       0xd1 obj/r_jump4.o
 .debug_abbrev  0x000035cc       0xd1 obj/r_jump5.o
 .debug_abbrev  0x0000369d       0xd1 obj/r_jump6.o
 .debug_abbrev  0x0000376e       0xd1 obj/r_jump7.o
 .debug_abbrev  0x0000383f       0xd1 obj/r_jump8.o
 .debug_abbrev  0x00003910       0xd1 obj/r_jump9.o
 .debug_abbrev  0x000039e1       0xd1 obj/r_jump10.o
 .debug_abbrev  0x00003ab2       0xd1 obj/r_attack1.o
 .debug_abbrev  0x00003b83       0xd1 obj/r_attack2.o
 .debug_abbrev  0x00003c54       0xd1 obj/r_attack3.o
 .debug_abbrev  0x00003d25       0xd1 obj/r_attack4.o
 .debug_abbrev  0x00003df6       0xd1 obj/r_attack5.o
 .debug_abbrev  0x00003ec7       0xd1 obj/r_attack6.o
 .debug_abbrev  0x00003f98       0xd1 obj/r_attack7.o
 .debug_abbrev  0x00004069       0xd1 obj/o_kihon001.o
 .debug_abbrev  0x0000413a       0xd1 obj/o_kihon002.o
 .debug_abbrev  0x0000420b       0xd1 obj/o_kihon003.o
 .debug_abbrev  0x000042dc       0xd1 obj/o_kihon004.o
 .debug_abbrev  0x000043ad       0xd1 obj/o_kihon005.o
 .debug_abbrev  0x0000447e       0xd1 obj/o_kihon006.o
 .debug_abbrev  0x0000454f       0xd1 obj/o_kihon007.o
 .debug_abbrev  0x00004620       0xd1 obj/o_kihon008.o
 .debug_abbrev  0x000046f1       0xd1 obj/o_kihon009.o
 .debug_abbrev  0x000047c2       0xd1 obj/o_kihon010.o
 .debug_abbrev  0x00004893       0xd1 obj/o_kougeki000.o
 .debug_abbrev  0x00004964       0xd1 obj/o_kougeki001.o
 .debug_abbrev  0x00004a35       0xd1 obj/o_kougeki002.o
 .debug_abbrev  0x00004b06       0xd1 obj/o_kougeki003.o
 .debug_abbrev  0x00004bd7       0xd1 obj/o_kougeki004.o
 .debug_abbrev  0x00004ca8       0xd1 obj/o_kougeki005.o
 .debug_abbrev  0x00004d79       0xd1 obj/o_kougeki006.o
 .debug_abbrev  0x00004e4a       0xd1 obj/o_kougeki007.o
 .debug_abbrev  0x00004f1b       0xd1 obj/o_kougeki008.o
 .debug_abbrev  0x00004fec       0xd1 obj/o_kougeki009.o
 .debug_abbrev  0x000050bd       0xd1 obj/o_kougeki010.o
 .debug_abbrev  0x0000518e       0xd1 obj/o_kougeki011.o
 .debug_abbrev  0x0000525f       0xd1 obj/o_kougeki012.o
 .debug_abbrev  0x00005330       0xd1 obj/o_kougeki013.o
 .debug_abbrev  0x00005401       0xd1 obj/o_kougeki014.o
 .debug_abbrev  0x000054d2       0xd1 obj/o_kougeki015.o
 .debug_abbrev  0x000055a3       0xd1 obj/o_kougeki016.o
 .debug_abbrev  0x00005674       0xd1 obj/o_kougeki017.o
 .debug_abbrev  0x00005745       0xd1 obj/o_kougeki018.o
 .debug_abbrev  0x00005816       0xd1 obj/o_kougeki019.o
 .debug_abbrev  0x000058e7       0xd1 obj/o_kougeki020.o
 .debug_abbrev  0x000059b8       0xd1 obj/o_yarare000.o
 .debug_abbrev  0x00005a89       0xd1 obj/o_yarare001.o
 .debug_abbrev  0x00005b5a       0xd1 obj/o_yarare002.o
 .debug_abbrev  0x00005c2b       0xd1 obj/o_yarare003.o
 .debug_abbrev  0x00005cfc       0xd1 obj/o_yarare004.o
 .debug_abbrev  0x00005dcd       0xd1 obj/o_yarare005.o
 .debug_abbrev  0x00005e9e       0xd1 obj/o_yarare006.o
 .debug_abbrev  0x00005f6f       0xd1 obj/o_yarare007.o
 .debug_abbrev  0x00006040       0xd1 obj/o_yarare008.o
 .debug_abbrev  0x00006111       0xd1 obj/o_yarare009.o
 .debug_abbrev  0x000061e2       0xd1 obj/o_yarare010.o
 .debug_abbrev  0x000062b3       0xd1 obj/o_yarare011.o
 .debug_abbrev  0x00006384       0xd1 obj/o_yarare012.o
 .debug_abbrev  0x00006455       0xd1 obj/o_yarare013.o
 .debug_abbrev  0x00006526       0xd1 obj/o_yarare014.o
 .debug_abbrev  0x000065f7       0xd1 obj/o_yarare015.o
 .debug_abbrev  0x000066c8       0xd1 obj/o_yarare016.o
 .debug_abbrev  0x00006799       0xd1 obj/o_yarare017.o
 .debug_abbrev  0x0000686a       0xd1 obj/o_yarare018.o
 .debug_abbrev  0x0000693b       0xd1 obj/o_yarare019.o
 .debug_abbrev  0x00006a0c       0xd1 obj/o_yarare020.o
 .debug_abbrev  0x00006add       0xca obj/o_fukiya000.o
 .debug_abbrev  0x00006ba7       0xca obj/awa.o
 .debug_abbrev  0x00006c71       0xd1 obj/ring_32_64_left.o
 .debug_abbrev  0x00006d42       0xd1 obj/ring_32_64_right.o
 .debug_abbrev  0x00006e13       0xd1 bg_parts/umia_.o
 .debug_abbrev  0x00006ee4       0xe2 bg_parts/umi_ab_256x512.o
 .debug_abbrev  0x00006fc6       0xe2 bg_parts/sango1024x256.o
 .debug_abbrev  0x000070a8       0xe2 bg_parts/sora.o
 .debug_abbrev  0x0000718a       0xe2 bg_parts/light4.o
 .debug_abbrev  0x0000726c       0xca bg_parts/wave2nd1.o
 .debug_abbrev  0x00007336       0xca bg_parts/wave2nd2.o
 .debug_abbrev  0x00007400       0xca bg_parts/wave2nd3.o

.debug_line     0x00000000     0x2f50
 *(.debug_line)
 .debug_line    0x00000000      0x386 main.o
 .debug_line    0x00000386      0xdad player.o
 .debug_line    0x00001133      0xae2 enemy.o
 .debug_line    0x00001c15      0xcdc bg.o
 .debug_line    0x000028f1      0x2ed hitcheck.o
 .debug_line    0x00002bde      0x372 ring.o

.debug_frame
 *(.debug_frame)

.debug_str
 *(.debug_str)

.debug_loc
 *(.debug_loc)

.debug_macinfo
 *(.debug_macinfo)

.debug_weaknames
 *(.debug_weaknames)

.debug_funcnames
 *(.debug_funcnames)

.debug_typenames
 *(.debug_typenames)

.debug_varnames
 *(.debug_varnames)

.stack          0x00080000        0x0
                0x00080000                _stack=.
 *(.stack)
OUTPUT(dolphin.elf elf32-littlearm)
